:020000040000FA
:040000000000702864
:080008006400A000030E0313C5
:100010008312A1000408A5000A08A2008A010B1996
:1000200014288C1A572867286400A80B1A287D30DA
:10003000A8005715A90B4B28FA30A900D81C3C285A
:10004000AA0B4B283C30AA00C20B4B288312031783
:100050000C308F0072308D00831603178C170C1430
:1000600000000000831203170C0803138312C20060
:100070003030C20258144128C20B41283C30C20023
:100080005814591F5328C803C808031D5328143097
:10009000C8005913D917571D53285711061E522847
:1000A000061241280616063081000B1167289818A1
:1000B0005F28181965281A08CA00DC146628181267
:1000C0001A081A081A08181666281A088C12220824
:1000D0008A0025088400210E8300A00E200E09004E
:1000E00055303002031D7528D62883015F30A000EB
:1000F0002130840064008001840AA00B7A284F30EC
:10010000A000A130840064008001840AA00B832831
:1001100083175F3090001130840064008001840AEE
:10012000900B8D285F309000913084006400800136
:10013000840A900B9628900190018301A001900100
:100140005530B000FA30A9007D30A8000530C80055
:100150008A150A1682218A110A12D81CC528831210
:1001600003170C308F0072308D00831603178C1725
:100170000C1400000000831203170C0803138312F1
:10018000C2003030C2025814C7283C30C20084017B
:10019000D6280313831606309F0000308500C03038
:1001A0008600C0308700031383120800B00164008A
:1001B000031383168C018D0106309F00833062008B
:1001C0000313831264008B138B1BE2280B11940121
:1001D0008C018D01860187011A081A081A0814304B
:1001E000C8005A106400C92012267C26A3260B17CB
:1001F0008B168B1776268E26A3266A26D715C7015F
:10020000C626D91F06295913D91376265818A825AA
:10021000591A0F29DC1C0129DC104B210129611816
:100220002B215818A8255F18A8256019A8258A1120
:100230000A1600208A110A12DA01DB01DC01DD0155
:10024000DE01DF01E001E101B901BA01BB01BC013E
:10025000BD01BE0101298B138B1B2B2961102826A0
:100260002E2634263A268A150A166F218A110A127A
:100270008A150A1682218A110A12D81C33295814A9
:100280005714E11430304302C2003C30AA008B17EF
:100290008B1F472908005A18592902304A02031DAA
:1002A00059295A145030C900A130A600CE01C4010A
:1002B000972D5A1C972D03304A02031D6C295B1F92
:1002C000882D59168616260884003E30031383169F
:1002D000800003138312972DDA188C294E08C7006B
:1002E0001F27D0004A02031D7829CE0AC40A972D81
:1002F000500898255C1C7F29CE0AC40A972D0A3025
:100300004A02031D8A2908304402031D8A29DA148F
:10031000C401972DC401882D5A199E294E08C70083
:100320001F27D0004A02031D9729CE0A972D0A30B5
:100330004A02031D9D295A15972D882DDA19C729C0
:100340004E08C7001F27D0004A02031DAA29CE0A63
:10035000C40A972D500898255C1CB129CE0AC40AFE
:10036000972D0A304A02031DBE2905304402031DA1
:10037000C529DA151530CE00C401972D2A30500258
:10038000031DC529CE0AC40A972DC401882D5A1A07
:10039000E8295D19DF294E08C7001F27D0004A024F
:1003A000031DD929CE0A3D305002031D972D5D153E
:1003B000972D500898255C1CDF29CE0A972D0A300E
:1003C0004A02031D972D5D1DE7295A16972D882D8A
:1003D000DA1A312ADC1A2A2A4E08C7001F27D00051
:1003E0004A02031D052ACE0AC40A3D305002031DED
:1003F000FB295C16972D2E305002031D972D1130CE
:100400004402031D302ADE17972D500898255C1CE6
:100410000C2ACE0AC40A972D0A304A02031D1B2A51
:1004200020305002031D302ACE0AC40ADA1650309A
:10043000CE00C401972D5C1E302A07304402031DF4
:10044000302A2A304A02031D302ADC165030CE00F2
:10045000C401972D0A304A02031D302ADA16972D5F
:10046000882D5A1B432A4E08C7001F27D0004A0276
:10047000031D3C2ACE0A972D0A304A02031D422A48
:100480005A17972D882DDA1BA92A4E08C7001F2757
:10049000D0004A02031D4F2ACE0AC40A972D5008E5
:1004A00098255C1C562ACE0AC40A972D0A304A02A7
:1004B000031D952A6019892AE0187B2A5F186D2A86
:1004C000601609304402031DA72ADA175F10E010F6
:1004D0006011C4011A30CE07972D0B304402031D62
:1004E000A72ADC1AA72ADA17C4016012E0106011EB
:1004F0000F30CE07972D0F304402031DA72ADC1AB8
:10050000A72ADA17C40160125F1060110730CE0706
:10051000972D0E304402031DA72ADC1AA72ADA17EA
:10052000C40160125F10E010972D5F189B2A5F14C2
:100530000930CE07452AE018A12AE0140430CE077E
:10054000452A6019A72A60150830CE07452AC4013C
:10055000882D5B18C22A4E08C7001F27D0004A0208
:10056000031DB42ACE0A972D0A304A02031DC12A60
:100570005B14E01CBE2AD030CE00972D8030CE0018
:10058000972D882DE018352B5C19B92B4E08C70024
:100590001F27D0004A02031DDA2ACE0AC40A3D30C2
:1005A0005002031D972D08304402031D342BE01721
:1005B000C401972D500898255C1CE12ACE0AC40A74
:1005C000972D0A304A02031D222B5C15DF18152BCC
:1005D0005E1A082BDC19FB2AED2A601E342B05302D
:1005E0004402031D342BDE16B030CE00DC115E1247
:1005F000DF10C401972D601E342B05304402031D0B
:10060000342BB030CE00DE125E12DF10C401972D05
:10061000601E342B09304402031D342BB030CE0051
:10062000DE12DC11DF10C401972D601A342B073065
:100630004402031D342BB030CE00DC115E12DE12FA
:10064000C401972DDC19282BDC150530CE07C62AEE
:100650005E1A2E2B5E160530CE07C62ADF18342B05
:10066000DF140930CE07C62A882DE01A522B4E0817
:10067000C7001F27D0004A02031D4B2BCE0AC40A15
:100680003D304A02031D972D08304402031D882D7A
:10069000E016C401972D500898255C1C882DCE0AC1
:1006A000C40A972DDB197D2B0A304A02031D712BDA
:1006B0001130D3004408D3020319612B0318612BB6
:1006C000882D26088400203003138316800003132E
:1006D0008312A60AD30B612BDB15C4010230D500AF
:1006E000972D260884004A080313831680000313FD
:1006F0008312A60AC903C40A972D61199A2B4E08C2
:10070000C7001F27D0004A02031D932BCE0AC40A3C
:100710003D304A02031D972D09304402031D882DE8
:100720006115C401972D500898255C1C882DCE0AB0
:10073000C40A972D611A7B2D0A304A02031DA92B8A
:10074000E11D882D6116E01C972DE01E972D611488
:10075000972DE119972D260884004A08C30003133A
:100760008316800003138312A60AC903C40AE11585
:10077000972DDF187B2D5B1B7B2DDB19FF2BDB18E7
:10078000E72B4E08C7001F27D0004A02031DD42BB9
:10079000CE0AC40A3D305002031D972D0530440295
:1007A000031DE62BDB14972D500898255C1CDB2BD2
:1007B000CE0AC40A972DDC19E62B5B1BE62B7D3095
:1007C0004A02031DE62B5B17C401972D882DDB1908
:1007D0007B2DBB300402031900000A304A02031DBE
:1007E000F42BDB15C401972D260884004A088312D8
:1007F0000317800003138312A60AC903972DDD187F
:10080000702C5B1A1F2CDD19702C4E08C7001F2797
:10081000D0004A02031D182CCE0AC40A3D305002F3
:10082000031D972D04304402031D462C5B16972DA3
:10083000500898255C1C3F2CCE0AC40A972DDB1A61
:100840003F2CDB1B322C0A304A02031D2E2CB9012F
:10085000BA01DB17DB16DD14C401972D4A08B90075
:10086000DB17972D0A304A02031D3B2CBA01DB1619
:10087000DD14C401972D4A08BA00DB16972D0A3003
:100880004A02031D472CDD14C401972D882DC4088E
:10089000031D462C63304A02031D4F2C6C2C433041
:1008A00098255C1C542C6C2C64304A02031D592C76
:1008B0006C2C443098255C1C5E2C6C2C61304A02F8
:1008C000031D632C6C2C413098255C1C682C6C2C0F
:1008D0007D304A02031D462CDD150430CE07C401CD
:1008E000DD1AD72C5C1B902C5D1AD72C4E08C70044
:1008F0001F27D0004A02031D892CCE0AC40A3D30AE
:100900005002031D972D07304402031DB72C5C17BE
:10091000972D500898255C1CB02CCE0AC40A972D40
:10092000DC1BB02C5D18A32C0A304A02031D9F2C3F
:10093000BB01BC015D14DC17DD16C401972D4A080C
:10094000BB005D14972D0A304A02031DAC2CBC017C
:10095000DC17DD16C401972D4A08BC00DC17972D63
:100960000A304A02031DB82CDD16C401972D882DCC
:10097000C408031DB72C64304A02031DC02CD32CBD
:10098000443098255C1CC52CD32C61304A02031DD1
:10099000CA2CD32C413098255C1CCF2CD32C7D3015
:1009A0004A02031DB72C5D16C4010730CE075D1B3C
:1009B000362D5E19F72CDE18362D4E08C7001F277E
:1009C000D0004A02031DF02CCE0AC40A3D3050026A
:1009D000031D972D06304402031D202D5E15972D13
:1009E000500898255C1C172DCE0AC40A972DDD1BD4
:1009F000172D5E180A2D0A304A02031D062DBD016F
:100A0000BE015E14DD175D17C401972D4A08BD00B5
:100A10005E14972D0A304A02031D132DBE01DD1707
:100A20005D17C401972D4A08BE00DD17972D0A30C7
:100A30004A02031D212D5E1D202D5D17C401972D37
:100A4000882DC408031D202D61304A02031D292D65
:100A5000322D413098255C1C2E2D322D7D304A02DE
:100A6000031D202DDE14C4010630CE075F1A7B2D36
:100A7000DF197B2D4E08C7001F27D0004A02031D37
:100A80004D2DCE0AC40A3D305002031D972D06306D
:100A90004402031D782D5F15972D500898255C1C86
:100AA000542DCE0AC40A972D0A304A02031D692D1F
:100AB0005F1D792D07304402031D882D642DC4016C
:100AC000DF155F16C401972DC401DF115F16C40145
:100AD000972D6018722D07304402031D792D601484
:100AE000CE0A3A2DC408031D882DDF15C4017B2DC5
:100AF000882DDF15C4015B1B832D7D304A02031D49
:100B0000972D5B17972D0A304A02031D882D972DCC
:100B1000DA01DB01DC01DD01DE01DF01E001E101E1
:100B2000B901BA01BB01BC01BE01BD01C40108008D
:100B30005C10A225D6004A08A2255602031DA12D4D
:100B40005C140800853E1A3E031C203E413E08000E
:100B50000230C000C1018C128B138B1BAC2D0526FB
:100B60000C1EAF2D02309900C008031DBD2D0526B7
:100B70000C1EB72D0A309900EF2D05260C1EBD2D39
:100B800041085F18CA2D6019CD2DD81CD02DDF1754
:100B90002E27D22D5F174C27D22DE0155B27D22DA3
:100BA000DF173D27CB0020304B020319ED2D6E30AF
:100BB0004B02031DE12D5E1FEB2D0A30CB005E13AF
:100BC000EB2D5C304B02031DE72D5E17BD2D7D30F4
:100BD0004B020319C0034B089900C10AB42D5F1FD3
:100BE000F42D5F105714FB2DE01DF92D60115714E3
:100BF000FB2D5810DF1305260C1EFB2D033099002A
:100C00008C168B178B1F012E0800FF30AF0064007D
:100C1000AF0B072E08000B3037020319102E080007
:100C2000D916080003138316193099009813181267
:100C300018131815981618108C160313831298178A
:100C400018139811181618111A081A081A0808000B
:100C500018308A0000208A110A12080018308A0011
:100C60003B208A110A12080018308A009E208A113F
:100C70000A12080019308A0034218A110A12080069
:100C800019308A0098218A110A12080019308A0046
:100C9000A6218A110A12080019308A00B0218A118F
:100CA0000A12080019308A00BA218A110A120800B3
:100CB00019308A00C4218A110A12080019308A00EA
:100CC000CE218A110A12080019308A00D8218A110F
:100CD0000A12080019308A00E2218A110A1208005B
:100CE00019308A00EC218A110A12080019308A0092
:100CF000F6218A110A1208001A308A0015228A1178
:100D00000A1208001A308A006D228A110A1208009D
:100D10001A308A0078228A110A1208001A308A00D2
:100D200082228A110A1208001A308A008C228A1143
:100D30000A12080010308A0000208A110A120800E6
:100D4000C601591008006400AC00FE30AB0064001E
:100D5000F930AB076400AB0BAA2EAC0BA72E00003A
:100D6000003408308A00450800208A11B200D919E1
:100D7000BF2E1A308A008C228A110A12C52EB21791
:100D80001A308A008C228A110A120800A0268B13BE
:100D90008B1BC62E4708C60009308A004608002172
:100DA0008A115918D52ED926CC2E8B178B1FD52EEC
:100DB0000800C5003E3C0319E52E45083C3C0319DC
:100DC000E72EB126C60A4608080059140800B70ADB
:100DD0000B26D91A762600304C02031DF12E46262A
:100DE0001C2F01304C02031DF72E4C261C2F023005
:100DF0004C02031DFD2E52261C2F03304C02031DF6
:100E0000032F58261C2F04304C02031D092F5E2689
:100E10001C2F05304C02031D0F2F64261C2F06309B
:100E20004C02031D152F6A261C2F07304C02031D90
:100E30001B2F70261C2F5226C60A46080800A02623
:100E40008B138B1B1F2F4E08C6000A308A004608E2
:100E500000228A118B178B1F2A2F0800A0268B13C4
:100E60008B1B2E2F4108C6000E308A004608002634
:100E70008A118B178B1F392F0800A0268B138B1B11
:100E80003D2F4108C6000F308A00460800278A110E
:100E90008B178B1F482F0800A0268B138B1B4C2F02
:100EA0004108C6000B308A00460800238A118B17C0
:100EB0008B1F572F0800A0268B138B1B5B2F41081D
:100EC000C6000C308A00460800248A118B178B1F3D
:100ED000662F0800FF30AE006400AE0B6C2F0800D8
:1010000082070B340B340B340B340B340B340B349E
:101010000B340B340B340B340B340B340B340B34D8
:101020000B340B340B340B340B340B340B340B34C8
:101030000B340B340B340B340B340B340B340B34B8
:101040000B340B340B340B340B340B340B340B34A8
:1010500029340B340B345F345E340B340A342734B8
:1010600028340034013402340334043405340634A3
:10107000073408340934263400340034783400341A
:1010800000340B340C340D340E340F34103411345E
:101090001234133414341534163417341834193404
:1010A0001A341B341C341D341E341F3420342134B4
:1010B00022342334243425340B340B340B340B34D6
:1010C0000B340B342A342B342C342D342E342F345F
:1010D00030343134323433343434353436343734D4
:1010E000383439343A343B343C343D343E343F3484
:1010F00040344134423443347C340B347D340B343B
:021100000B34AE
:101200008207783450344C3420344D346534733490
:10121000733461346734653420344434693473344E
:1012200070346C34613479342034503472346F3417
:101230006734723461346D343C34203420342034CB
:101240002034203420342034203444346534733442
:10125000693467346E34653464342034423479340C
:101260003C3420342034203420342034413472344F
:101270006D34613467346834203445346C346534FB
:101280006334743472346934633461346C343C34A0
:1012900020342034203420342034563465347234E1
:1012A000733469346F346E34203431342E34303436
:1012B00065343E3443346F346E3466346934673495
:1012C000753472346134743469346F346E3420345C
:1012D0004C3469347334743420345234653471348A
:1012E00075346534733474343E3443346F346E343F
:1012F00066346934673475347234613474346934F3
:101300006F346E34203452346534733470346F3437
:101310006E34733465343E3443347534723472340D
:1013200065346E347434203443346F346E34663430
:1013300069346734753472346134743469346F34A9
:101340006E3420345234653471342E343E342034BB
:101350004834653461347234743420346234653412
:101360006134743420346D346534733473346134CF
:101400008207783470346C342D3463346D346E3428
:0E14100064347B3468346F3470343D342A34D5
:06142A00203473346F341E
:1014300075347234633465343D34743461347234D9
:101440006734653474343D346134653463342D3429
:10145000743476346F34733464342E3464346534C5
:101460006634613475346C34743420342034203460
:0E147000203420342034203420342034203422
:1014A00020347D346F34733464342E3462346134C8
:1014B00073346934633463346F346E34663469343E
:1014C00067342E346C346934733474347234653454
:1014D000733470346F346E347334653463347534FC
:0C14E0007234723465346E3474347B3422
:10150000203463346F346D346D3461346E3464343C
:101510003D3463346C3465346134723477347234FE
:101520006934743465346534783463346C347534B8
:101530007334693476346534723465347134753497
:06154000653473347434BD
:10156000203474346534783474343D3472346F34D8
:1015700077343D3463346F346C3475346D346E3489
:101580003D34643465346C34613479343D346134D1
:101590006C346534723474343D3479346E347D3453
:1015A00020346E346534773463346F346E3466348B
:1015B0003D3469346E347434653472347634613455
:0415C0006C343D3416
:101600008207783470346C342D347334743461341C
:1016100074340A347B340A3468346F3470343D34A3
:1016200031340A3473346F3475347234633465344E
:101630003D346134653463342D34743476346F341E
:10164000733464342E3464346534663461347534F0
:101650006C3474342034203420342034203420344A
:101660002034203420340A347434613472346734C2
:10167000653474343D342A340A347D340A34633496
:101680006F346E346634693467342E346C346934A4
:10169000733474340A347B340A34723465346334FA
:1016A0006F346E3466343D346E346534773463346D
:1016B0006F346E3466340A347234653463346F3494
:1016C0006E3466343D3469346E3474346534723447
:0C16D000763461346C340A347D340A3402
:101800008207783470346C342D347334743461341A
:1018100074340A347B340A3468346F3470343D34A1
:1018200031340A3473346F3475347234633465344C
:101830003D346134653463342D34743476346F341C
:10184000733464342E3464346534663461347534EE
:101850006C34743420342034203420342034203448
:101860002034203420340A347434613472346734C0
:10187000653474343D342A340A347D340A34633494
:101880006F346E346634693467342E34633475349F
:101890007234723465346E3474340A347B340A34EE
:1018A0006E346534773463346F346E3466343D346B
:1018B000643465346634613475346C347434203483
:1018C0002034203420342034203420342034203478
:1018D0000A3469346E347434653472347634613465
:0C18E0006C343D3435340A347D340A3455
:101C00008207783470346C342D3473347434613416
:101C100074340A347B340A3468346F3470343D349D
:101C200031340A3473346F34753472346334653448
:101C30003D346134653463342D34743476346F3418
:101C4000733464342E3464346534663461347534EA
:101C50006C34743420342034203420342034203444
:101C60002034203420340A347434613472346734BC
:101C7000653474343D342A340A347D340A3468348B
:101C800062346534613474342E34623461347334B4
:101C9000693463340A347B340A3469346E347434FE
:101CA00065347234763461346C343D3435340A34FE
:041CB0007D340A3441
:101E00008207783470346C342D3473347434613414
:101E100074340A347B340A3468346F3470343D349B
:101E200031340A3473346F34753472346334653446
:101E30003D346134653463342D34743476346F3416
:101E4000733464342E3464346534663461347534E8
:101E50006C34743420342034203420342034203442
:101E60002034203420340A347434613472346734BA
:101E7000653474343D342A340A347D340A3463348E
:101E80006F346E346634693467342E3462346134AE
:101E90007334693463340A347B340A3469346E34FD
:101EA000743465347234763461346C343D34353492
:061EB0000A347D340A34FF
:102000000B135912DC190B288A150A16F6218A11AE
:102010000A16571811288A150A1682228A110A16DA
:102020004B2857105F1F25285F13BF010530B700ED
:102030008A150A16BA218A110A165930C7008A1160
:102040000A12C6268A110A167529E11C3828E110E1
:10205000BF010530B7008A150A16BA217430C700CF
:102060008A110A168A110A12C6268A110A167529B9
:10207000E01D7529E011BF010530B7008A150A1669
:10208000BA218A110A168B30C7008A110A12C62695
:102090008A110A167529BC08031D5C28BB08031D9C
:1020A00052285A2830303B02031D57285A28BF00B7
:1020B000BF038628BF0186283030BB02031D692874
:1020C0003030BC02BC0803195A283C08BF00BF03CB
:1020D000862802303B02031D6E28742803185A28F4
:1020E00001303B02031981283030BC0213303C0719
:1020F000BF001B303F02031D7E28862803185A2884
:1021000086283030BC0209303C07BF00BA08031DE6
:10211000A228B908031D8D289A2830303902031DE2
:1021200092289A28B700B7038A150A16E2218A1165
:102130000A16C9280530B7008A150A16E2218A1145
:102140000A16C9283030B902031DB02830303A02CF
:10215000B700B7038A150A16E2218A110A16C928A0
:102160003030BA0201303902031DBA28BA08031D03
:10217000BA28C2280A30B7008A150A16E2218A1145
:102180000A16C9280930B7008A150A16E2218A11F1
:102190000A16BE08031DDD28BD08031DD028D92856
:1021A00030303D02031DD62859132E295917C80077
:1021B0002E291430C80059172E293030BD02031DB6
:1021C000EA283030BE02BE0803192E293E08C80096
:1021D00059172E293030BE0201303D02031DF3286D
:1021E0000A30BD002A2902303D02031DFA281430AE
:1021F000BD002A2903303D02031D01291E30BD0008
:102200002A2904303D02031D08292830BD002A294F
:1022100005303D02031D0F293230BD002A2906304A
:102220003D02031D16293C30BD002A2907303D021E
:10223000031D1D294630BD002A2908303D02031D1B
:1022400024295030BD002A2909303D02031DD92818
:102250005A30BD003D083E07C8005917DF1937291D
:10226000D9158A150A16CE218A110A163C298A1513
:102270000A16E2218A110A165030CF00A1308400DC
:1022800003138316000803138312C5003E3C031991
:10229000752945085C3C03195F29DE1D582945084E
:1022A0006E3C0319622945084E3C03196229DE1170
:1022B0008A110A12B1268A110A16840A7329DE15B8
:1022C000840A7329DE11B70ADF1D6C298A150A16E4
:1022D000E2218A110A167229D9158A150A16CE2109
:1022E0008A110A16840ACF0B4029D9115030CF0029
:1022F000A1308400030103138316800003138312AB
:10230000840ACF0B7A290B170B1F8329861208002A
:10300000A13084001130D2008B138B1B0028831257
:1030100003170A308F002E308D0034308E000313DA
:1030200083122E30D1006400831603178C181328E6
:10303000831203178D0003138316000803138312F2
:10304000831203178C00831603178C170C15553049
:103050008D00AA308D008C14000000000313831231
:10306000840AD10A5108D20B1328831603170C11B6
:10307000031383120800A13084001030D2008B1398
:103080008B1B3B28831203170E308F0023308D00DB
:1030900034308E00031383122330D1006400831672
:1030A00003178C184E28831203178D000313831601
:1030B000000803138312831203178C00831603176F
:1030C0008C170C1555308D00AA308D008C14000023
:1030D000000003138312840AD10A5108D20B4E2830
:1030E000840A831203170E308F0056308D0034305F
:1030F0008E00031383125630D10064008316031729
:103100008C187D28831203178D0003138316000883
:1031100003138312831203178C00831603178C1773
:103120000C1555308D00AA308D008C140000000065
:10313000831603170C11031383120800A1308400B7
:103140001030D2008B138B1B9E28831203170C3078
:103150008F0023308D0034308E0003138312233010
:10316000D1006400831603178C18B128831203174B
:103170008D000313831600080313831283120317B1
:103180008C00831603178C170C1555308D00AA3050
:103190008D008C140000000003138312840AD10AEE
:1031A0005108D20BB1286400A13084001030D20045
:1031B000831203170C308F0058308D0034308E008E
:1031C000031383125830D1006400831603178C1840
:1031D000E428831203178D000313831600080313DA
:1031E0008312831203178C00831603178C170C1598
:1031F00055308D00AA308D008C14000000000313A0
:103200008312840AD10A5108D20BE428840A83125B
:1032100003170C308F0072308D0034308E00031392
:1032200083127230D1006400831603178C1813299F
:10323000831203178D0003138316000803138312F0
:10324000831203178C00831603178C170C15553047
:103250008D00AA308D008C14000000008316031727
:103260000C11031383120800A13084001030D20027
:103270008B138B1B3429831203170B308F002330E1
:103280008D0034308E00031383122330D10064008C
:10329000831603178C184729831203178D00031315
:1032A0008316000803138312831203178C008316FE
:1032B00003178C170C1555308D00AA308D008C1417
:1032C0000000000003138312840AD10A5108D20BB4
:1032D0004729831603170C11031383120800831266
:1032E000031703018D00AA308C00831603178C137B
:1032F0000C1555308D00AA308D008C140C11031361
:10330000831208008312031703018D00831603172D
:103310008C130C14831203170C0803138312D400AC
:10332000AA305402031D9629D8140800D8100800AA
:10333000D91C9D29051E9F29A529051EA5295915BA
:10334000D91CA429D910A529D91408003708B1001F
:103350003F08B2008C221830B1000030CC000800C9
:103360003708B1003F08B2008C221930B10001309B
:10337000CC0008003708B1003F08B2008C221A3098
:10338000B1000230CC0008003708B1003F08B2009D
:103390008C221B30B1000330CC0008003708B1008C
:1033A0003F08B2008C221C30B1000430CC00080071
:1033B0003708B1003F08B2008C221D30B100053043
:1033C000CC0008003708B1003F08B2008C221E3044
:1033D000B1000630CC0008003708B1003F08B20049
:1033E0008C221F30B1000730CC0008001D30B60021
:1033F000B701B101B2018C221F30B1000B30B20015
:103400008C22B60BFE29B70A0C3037020319112A99
:103410003708B100B2018C221F30B1001D30B60058
:10342000FE29D912B701BA2108003030B100B2012B
:103430008C223030B100B2018C22DB30B200B101FD
:103440008C221030B100B2018C22D918432ACC3022
:10345000B200B1018C221030B100B2018C221230C6
:10346000B100B2018C221330B100FA30B2008C22CC
:103470001A30B1001430B2008C221830B10036304E
:10348000B2008C225E2ACC30B200B1018C22103006
:10349000B100B2018C221230B100B2018C221B307B
:1034A000B100D130B2008C221A30B1001430B20019
:1034B0008C221830B1003630B2008C22C030B200FD
:1034C000B1018C220C30B3001830B100E030B200F2
:1034D0008C22B30B642A59110800CE30B200B1011E
:1034E0008C221330B100FA30B2008C220710080091
:1034F000CE30B200B1018C221B30B100FE30B200E0
:103500008C220800CE30B200B1018C221B30B100F9
:10351000D530B2008C2208000830B4008716871519
:103520008714871687103108B5009D220830B40033
:103530003208B5009D22871408006400B4080319FE
:10354000B62AB51FA52A8716A62A87120A30AD000B
:103550006400AD0BA82A87110A30AD006400AD0BE2
:10356000AE2A8715B4030310B50D9D2A08000A3052
:0A357000AD006400AD0BB92A08009D
:00000001FF
